:100000000C9463000C948B000C948B000C948B006C
:100010000C948B000C948B000C948B000C948B0034
:100020000C948B000C9421010C948B000C948B008D
:100030000C948B000C948B000C948B000C948B0014
:100040000C9459120C948B000C948B000C948B0024
:100050000C948B000C948B000C948B000C948B00F4
:100060000C948B000C948B000000000024002700EF
:100070002A0000000000250028002B0000000000DE
:1000800023002600290004040404040404040202DA
:100090000202020203030303030301020408102007
:1000A0004080010204081020010204081020000012
:1000B0000008000201000003040700000000000027
:1000C00000008D0A4C1211241FBECFEFD8E0DEBF16
:1000D000CDBF11E0A0E0B1E0E2ECF6E402C0059093
:1000E0000D92AA3AB107D9F722E0AAEAB1E001C01D
:1000F0001D92A739B207E1F710E0C3E6D0E004C0D3
:100100002197FE010E945420C136D107C9F70E94F1
:10011000731D0C945F230C940000CF93DF9300D0E9
:10012000CDB7DEB79A83898389819A81FC011082D9
:1001300089819A819093AB018093AA0189819A81E8
:100140000E94AF001092B5011092B4011092AD015F
:100150001092AC010F900F90DF91CF910895CF9343
:10016000DF9300D000D000D0CDB7DEB79E838D8363
:1001700019821A821B821C8280E790E0FC01208198
:1001800080E790E02E7FFC01208380E790E0FC0177
:10019000208180E790E0297FFC01208386EB90E0BE
:1001A000FC01208186EB90E02F7DFC01208381EB18
:1001B00090E0FC01208181EB90E02460FC01208331
:1001C00081EB90E0FC01208181EB90E02C7FFC0131
:1001D000208380E090E0A0E8B2E489839A83AB8337
:1001E000BC8380EB90E0FC01208180EB90E02C7FD1
:1001F000FC01208381EB90E0FC01208181EB90E009
:10020000277FFC01208329813A814B815C8161E059
:1002100070E08AE796E40E94FF1DDC01CB01BC017F
:10022000CD010E94711EDC01CB0181958093B30149
:1002300026960FB6F894DEBF0FBECDBFDF91CF91EB
:1002400008951F920F920FB60F9211242F933F9390
:100250004F935F936F937F938F939F93AF93BF93CE
:10026000EF93FF93CF93DF931F92CDB7DEB782EB6F
:1002700090E02091B301FC0120838091B401909122
:10028000B50101969093B5018093B4018091AC01C2
:100290009091AD0121E0892B09F420E0222309F49B
:1002A0008CC08091AE019091AF01A091B001B0914E
:1002B000B1010197A109B1098093AE019093AF01FB
:1002C000A093B001B093B1018091AE019091AF01C4
:1002D000A091B001B091B10121E0181619061A06DB
:1002E0001B060CF420E0222309F467C08091B201C0
:1002F000181654F48091B4019091B5010196883E8E
:10030000934014F481E001C080E0882319F18091CA
:10031000AC019091AD019C01990F440B550B80E00D
:100320009FE2ADE0B0E0BC01CD010E94F41FDA0114
:10033000C9018093AE019093AF01A093B001B09337
:10034000B1018091B4019091B50101969093B501EE
:100350008093B4018091B20188234CF48091B40160
:100360009091B5010197992314F081E001C080E0DC
:10037000882319F18091AC019091AD019C01990FF6
:10038000440B550B80E09FE2ADE0B0E0BC01CD0135
:100390000E94F41FDA01C9018093AE019093AF016E
:1003A000A093B001B093B1018091B4019091B501D7
:1003B00001979093B5018093B4018091B40190911D
:1003C000B50121E0883E93400CF420E0222309F49B
:1003D00080C01092B5011092B4018091B8018F5F76
:1003E0008093B8019091B80181E09C3308F480E0DB
:1003F000882309F46EC01092B8018091B7018F5F15
:100400008093B7019091B70181E09C3308F480E0BC
:10041000882309F45EC01092B7018091B6018F5F06
:100420008093B6019091B60181E0983108F480E0A4
:10043000882309F44EC01092B6018091B9018F5FF4
:100440008093B9019091BA0181E0923009F080E087
:10045000882381F08091AA019091AB0160E070E067
:100460000E948C03882319F08DE189830DC08CE1F3
:1004700089830AC08091BA01882F90E0019780504B
:100480009F4FFC01808189839091B90181E029818E
:10049000291708F080E08823E1F081E08093B9011A
:1004A0008091BA018F5F8093BA019091BA0181E087
:1004B0009D3008F480E0882361F081E08093BA01E8
:1004C0008091BB019091BC0101969093BC018093F7
:1004D000BB010F90DF91CF91FF91EF91BF91AF9151
:1004E0009F918F917F916F915F914F913F912F914C
:1004F0000F900FBE0F901F901895CF93DF9300D0F1
:1005000000D01F92CDB7DEB79A8389836B834C836B
:100510002D838B81883110F080E014C08C818C3366
:1005200010F080E00FC08D818C3310F080E00AC0A5
:100530008B818093B6018C818093B7018D818093EC
:10054000B80181E00F900F900F900F900F90DF9106
:10055000CF910895CF93DF9300D000D000D0CDB7D6
:10056000DEB79A8389836B834C833E832D838B8193
:10057000882319F08B81803210F080E01BC08C81C1
:10058000882319F08C818D3010F080E013C08D81AC
:100590009E81992314F480E00DC08B818093B90172
:1005A0008C818093BA018D819E819093BC01809350
:1005B000BB0181E026960FB6F894DEBF0FBECDBF1B
:1005C000DF91CF910895CF93DF9300D0CDB7DEB701
:1005D0009A83898389819A810E94AF001092B50124
:1005E0001092B40182EB90E02091B301FC012083D2
:1005F00080E790E0FC01208180E790E02160FC0131
:1006000020838FE590E0FC0120818FE590E0206859
:10061000FC01208389819A8121E0FC0120830F90D5
:100620000F90DF91CF910895CF93DF9300D0CDB796
:10063000DEB79A83898380E790E0FC01208180E720
:1006400090E02E7FFC0120838FE590E0FC0120816B
:100650008FE590E02F77FC01208389819A81FC014E
:1006600010820F900F90DF91CF910895CF93DF9379
:1006700000D0CDB7DEB79A8389838091B8010F90FF
:100680000F90DF91CF910895CF93DF9300D0CDB736
:10069000DEB79A8389838091B7010F900F90DF9125
:1006A000CF910895CF93DF9300D0CDB7DEB79A8373
:1006B00089838091B6010F900F90DF91CF910895BB
:1006C000CF93DF9300D0CDB7DEB79A838983809133
:1006D000B9010F900F90DF91CF910895CF93DF93E1
:1006E00000D0CDB7DEB79A8389838091BA010F908D
:1006F0000F90DF91CF910895CF93DF9300D0CDB7C6
:10070000DEB79A8389838091BB019091BC010F90E1
:100710000F90DF91CF910895CF93DF9300D000D059
:10072000CDB7DEB79A8389837C836B838B819C8171
:10073000892B31F48091BB019091BC019C838B8308
:100740008B819C8183709927892B49F48B819C81B3
:1007500024E630E0B9010E94E01F892B49F48B8127
:100760009C8120E931E0B9010E94E01F892B11F43E
:1007700081E001C080E00F900F900F900F90DF910B
:10078000CF910895CF92DF92EF92FF920F931F9334
:10079000CF93DF93CDB7DEB729970FB6F894DEBFBE
:1007A0000FBECDBF9F838E837987688719821A8297
:1007B0001B821C8288859985892B29F482EB97E01E
:1007C0009987888722C0888599858C3697402CF434
:1007D0008CE697E09987888718C088859985833B40
:1007E00097402CF082EB97E0998788870EC0888528
:1007F00099858C36974049F088859985823B97404A
:1008000021F082EB97E0998788878E819F810E94F3
:100810007C039C0188859985A901481B590BCA0155
:10082000092E000CAA0BBB0BBC01CD010E94A91E16
:10083000DC01CB0120E03FE946EB53E4BC01CD01F4
:100840000E945E1FDC01CB016C017D0169817A8110
:100850008B819C810E94A71EDC01CB019C01AD0114
:10086000C701B6010E948E1DDC01CB01BC01CD0188
:100870000E94781EDC01CB0189839A83AB83BC8301
:100880001D828D81082F10E08E819F810E946E0352
:10089000882F90E0019721E0081719070CF020E05D
:1008A0002223D9F08D81882F90E080509F4FFC014A
:1008B0008081882F90E0A0E0B0E029813A814B81CF
:1008C0005C81820F931FA41FB51F89839A83AB831A
:1008D000BC838D818F5F8D83D4CF8E819F810E9459
:1008E0006003282F30E040E050E089819A81AB819D
:1008F000BC81280F391F4A1F5B1FDA01C901880F0D
:10090000991FAA1FBB1F820F931FA41FB51F880F1B
:10091000991FAA1FBB1F880F991FAA1FBB1F880FF3
:10092000991FAA1FBB1F89839A83AB83BC838E81C7
:100930009F810E945203282F30E040E050E08981DF
:100940009A81AB81BC81280F391F4A1F5B1F8CE342
:1009500090E0DC010E943520DC01CB0189839A8381
:10096000AB83BC838E819F810E944403282F30E09B
:1009700040E050E089819A81AB81BC81280F391F0A
:100980004A1F5B1F8CE390E0DC010E943520DC01F4
:10099000CB0189839A83AB83BC838E819F810E9424
:1009A0003603882F90E0A0E0B0E029813A814B81A6
:1009B0005C81820F931FA41FB51F89839A83AB8329
:1009C000BC8389819A81AB81BC8180329940AC4BD8
:1009D000B84360F089819A81AB81BC8180589E4A7E
:1009E000AE4FBF4F89839A83AB83BC838E819F8137
:1009F0000E947C039C018E819F81B9010E948C031F
:100A00008823B9F08E819F810E946E03982F81E028
:100A1000933008F080E0882361F089819A81AB816E
:100A2000BC8180589145A140B10989839A83AB83E9
:100A3000BC8389819A81AB81BC8180589145A1405A
:100A4000B109BC01CD0129960FB6F894DEBF0FBEE7
:100A5000CDBFDF91CF911F910F91FF90EF90DF906D
:100A6000CF900895CF93DF9300D000D000D0CDB7C2
:100A7000DEB79A8389834B835C836D837E8320E01A
:100A800030E040E251E46B817C818D819E810E9447
:100A90005E1FDC01CB01BC01CD010E94711EDC0197
:100AA000CB019C0189819A81B9010E94600526963B
:100AB0000FB6F894DEBF0FBECDBFDF91CF91089582
:100AC000CF93DF9300D000D0CDB7DEB79A83898370
:100AD0007C836B838B819C8180339F4D2CF08B8139
:100AE0009C81813D904214F080E09CC08B819C8170
:100AF0009093AD018093AC018091AC019091AD01D8
:100B000021E0892B09F020E0222359F01092AE0158
:100B10001092AF011092B0011092B1011092B20187
:100B200080C08091AC019091AD019C01990F440B64
:100B3000550B80E09FE2ADE0B0E0BC01CD010E942A
:100B4000F41FDA01C901892B8A2B8B2B99F0809134
:100B5000AC019091AD019C01990F440B550B80E0C5
:100B60009FE2ADE0B0E0BC01CD010E94F41FDA01CC
:100B7000C90119C08091AC019091AD019C01990F00
:100B8000440B550B80E09FE2ADE0B0E0BC01CD012D
:100B90000E94F41FDA01C901B095A0959095819546
:100BA0009F4FAF4FBF4F8093AE019093AF01A09383
:100BB000B001B093B1014091AC015091AD01809171
:100BC000AC019091AD01181619064CF08091AC0162
:100BD0009091AD0122273327281B390B04C02091A7
:100BE000AC013091AD01CA01B9010E94E01FCB01F7
:100BF0008093B2018091AC019091AD011816190655
:100C000044F08091AC019091AD019195819591094D
:100C100004C08091AC019091AD019093AD0180939F
:100C2000AC0181E00F900F900F900F90DF91CF916A
:100C30000895CF93DF9300D0CDB7DEB79A83898331
:100C40008091B201282F880F330B8091AC019091D5
:100C5000AD01289FA001299F500D389F500D1124F0
:100C6000CA010F900F90DF91CF910895CF92DF923C
:100C7000EF92FF921F93CF93DF93CDB7DEB76997C3
:100C80000FB6F894DEBF0FBECDBF9B8B8A8B4C8B0B
:100C90005D8B6E8B7F8B398F288F8C899D89AE8978
:100CA000BF8920E831E541E050E0BC01CD010E9460
:100CB000F41FDA01C90189839A83AB83BC838981DC
:100CC0009A81AB81BC819C01AD0160E871E581E056
:100CD00090E00E94D01F9B01AC018C899D89AE8958
:100CE000BF89821B930BA40BB50BBC01CD010E94E5
:100CF000A71EDC01CB018C879D87AE87BF876981EA
:100D00007A818B819C810E94A71EDC01CB0120E0AF
:100D10003FE946EB53E4BC01CD010E94FF1DDC011D
:100D2000CB01BC01CD010E94711EDC01CB019E8371
:100D30008D8369817A818B819C810E94A71E6B01C2
:100D40007C018D819E81092E000CAA0BBB0BBC017E
:100D5000CD010E94A91EDC01CB0120E03FE946EB5A
:100D600053E4BC01CD010E945E1FDC01CB019C015C
:100D7000AD01C701B6010E948D1DDC01CB018F833F
:100D80009887A987BA87888D998D892B29F482EB5A
:100D900097E0998F888F22C0888D998D8C369740E7
:100DA0002CF48CE697E0998F888F18C0888D998DE8
:100DB000833B97402CF082EB97E0998F888F0EC091
:100DC000888D998D8C36974049F0888D998D823B1E
:100DD000974021F082EB97E0998F888F2D813E819B
:100DE000888D998D820F931F9E838D8320E03FE92C
:100DF00046EB53E46F81788589859A850E94591F57
:100E0000882314F081E0E6C12D813E81888D998D83
:100E10002817390714F482E0DDC11B868B85882FE3
:100E200090E080509F4FFC018081882F90E0092E38
:100E3000000CAA0BBB0BBC01CD010E94A91EDC015A
:100E4000CB0111E09C01AD016F81788589859A8580
:100E50000E94591F18160CF010E0112309F446C027
:100E60008B85882F90E080509F4FFC018081882FD8
:100E700090E0092E000CAA0BBB0BBC01CD010E9417
:100E8000A91EDC01CB019C01AD016F8178858985AC
:100E90009A850E948D1DDC01CB018F839887A987DD
:100EA000BA878B85813059F42D813E818A899B894F
:100EB000B9010E948C03882311F081E001C080E019
:100EC000882381F020E030E040E85FE36F8178859F
:100ED00089859A850E948D1DDC01CB018F839887BF
:100EE000A987BA878B858F5F8B8798CF8B858F5F1C
:100EF0008B878B858D3038F081E08B878D819E814B
:100F000001969E838D8320E030EC48EA57E46F81A0
:100F1000788589859A850E94591F882314F084E07A
:100F200059C16F81788589859A850E94781EDC0178
:100F3000CB0189839A83AB83BC8369817A818B815E
:100F40009C810E94A71EDC01CB019C01AD016F8139
:100F5000788589859A850E948D1DDC01CB0120E072
:100F600030E0A901BC01CD010E94591F18165CF4A4
:100F700089819A81AB81BC810196A11DB11D8983B4
:100F80009A83AB83BC8320E030E041E655E46C8576
:100F90007D858E859F850E94FF1DDC01CB01BC01F4
:100FA000CD010E94781EDC01CB01888B8889282F17
:100FB00030E040E050E080E19EE0DC010E9435201E
:100FC000DC01CB01BC01CD010E94A71EDC01CB01DD
:100FD0009C01AD016C857D858E859F850E948D1D50
:100FE000DC01CB018C879D87AE87BF8720E030E096
:100FF00041E655E46C857D858E859F850E94591F4D
:10100000882314F085E0E6C020E030E040E752E4B9
:101010006C857D858E859F850E94FF1DDC01CB013F
:10102000BC01CD010E94781EDC01CB01898B89892E
:10103000282F30E040E050E08CE390E0DC010E949B
:101040003520DC01CB01BC01CD010E94A71EDC01D3
:10105000CB019C01AD016C857D858E859F850E94AD
:101060008D1DDC01CB018C879D87AE87BF8720E07B
:1010700030E040E752E46C857D858E859F850E9437
:10108000591F882314F086E0A5C08D819E8190931E
:10109000BC018093BB018B858093BA0189818093C9
:1010A000B9018091B9018F3131F48091BA018C304E
:1010B00011F481E001C080E0882399F08091BB01A8
:1010C0009091BC019C012F5F3F4F8A899B89B90198
:1010D0000E948C03882329F08D819E8101969E8336
:1010E0008D832D813E818A899B89B9010E948C0361
:1010F000882309F45EC08091B9018F5F8093B901A4
:101100008091BA018230A9F48091BA01882F90E0D1
:10111000019780509F4FFC018081882F90E00196BD
:10112000092E000CAA0BBB0B89839A83AB83BC836B
:1011300011C08091BA01882F90E0019780509F4F95
:10114000FC018081882F90E0A0E0B0E089839A8341
:10115000AB83BC838091B901882F90E0A0E0B0E020
:1011600061E029813A814B815C81281739074A0760
:101170005B0708F060E06623E1F081E08093B9014D
:101180008091BA018F5F8093BA019091BA0181E09A
:101190009D3008F480E0882361F081E08093BA01FB
:1011A0008091BB019091BC0101969093BC0180930A
:1011B000BB0188898093B60189898093B7016C85CA
:1011C0007D858E859F850E94781EDC01CB018093F2
:1011D000B80180E069960FB6F894DEBF0FBECDBFB0
:1011E000DF91CF911F91FF90EF90DF90CF90089506
:1011F000CF93DF9300D000D000D0CDB7DEB79A8375
:1012000089834B835C836D837E838B819C81AD81DD
:10121000BE8120E831E541E050E0BC01CD010E94F3
:10122000F41FDA01C9010496A11DB11D27E030E0C9
:1012300040E050E0BC01CD010E94F41FDC01CB0175
:1012400026960FB6F894DEBF0FBECDBFDF91CF91CB
:101250000895CF93DF9300D0CDB7DEB79A8389830B
:1012600089819A8160E070E00E94C2039B01AC0119
:1012700089819A81BA01A9010E94F8080F900F9004
:10128000DF91CF910895CF93DF93CDB7DEB762E0C2
:1012900082E00E946C1461E083E00E946C1461E0C3
:1012A00084E00E946C1461E085E00E946C1461E0AF
:1012B00086E00E946C1461E087E00E946C1461E09B
:1012C00088E00E946C1461E089E00E946C1461E087
:1012D0008AE00E946C1461E08BE00E946C1461E073
:1012E0008CE00E946C1461E08DE00E946C148CED27
:1012F00091E00E94140324EE37E048E067E18CEDB2
:1013000091E00E94AA0220E045E26DE08CED91E0C0
:101310000E947D028CED91E00E94E302DF91CF916B
:101320000895CF93DF93CDB7DEB72C970FB6F8941F
:10133000DEBF0FBECDBF9C878B8789E090E09A8788
:1013400089871A82198289819A8105975CF489813B
:10135000875F61E00E94921589819A8101969A8344
:101360008983F1CF62E370E080E090E00E94541343
:101370001C821B828B819C8105975CF48B81875F2B
:1013800060E00E9492158B819C8101969C838B83E7
:10139000F1CF1E821D828D819E810497BCF48B85C6
:1013A0009C850D8002C0959587950A94E2F781701F
:1013B0009927892B29F08D81875F61E00E94921522
:1013C0008D819E8101969E838D83E5CF68EE73E0CB
:1013D00080E090E00E94541318861F828F819885C8
:1013E00004975CF48F81875F60E00E9492158F8183
:1013F0009885019698878F83F1CF2C960FB6F89435
:10140000DEBF0FBECDBFDF91CF910895CF93DF93A5
:1014100000D0CDB7DEB71A82198289819A810697EA
:10142000B4F42091DA013091DB0189819A81820F35
:10143000931FFC018081082E000C990BC0970E941D
:10144000910989819A8101969A838983E6CF0F90C9
:101450000F90DF91CF910895CF93DF9300D000D00C
:10146000CDB7DEB782E00E94191621E0019709F09E
:1014700020E02223B9F761E08DE00E94921560E040
:1014800070E08CED91E00E94C203DC01CB01898306
:101490009A83AB83BC8389819A81AB81BC81AC0187
:1014A000BD018DEB91E00E94F50A9093DB018093E2
:1014B000DA0160E08DE00E9492150E94060A0F900A
:1014C0000F900F900F90DF91CF910895CF93DF93FE
:1014D00000D000D0CDB7DEB79A8389837C836B833D
:1014E00089819A81019791F48B819C81019671F495
:1014F0002EE130E048E050E06CE071E08DEB91E0EF
:101500000E949A0A8CED91E00E948D000F900F903E
:101510000F900F90DF91CF910895CF93DF93CDB7C8
:10152000DEB76FEF7FEF81E090E00E94660ADF9107
:10153000CF910895CF93DF93CDB7DEB728970FB63D
:10154000F894DEBF0FBECDBF9A8389837C836B8303
:101550005E834D8338872F8389819A812B813C81DB
:10156000FC013183208389819A812D813E81FC0198
:101570003383228389819A812F813885FC013583C9
:10158000248328960FB6F894DEBF0FBECDBFDF913F
:10159000CF910895CF93DF9300D000D000D0CDB786
:1015A000DEB79A8389837C836B835E834D838981D5
:1015B0009A812B813C81FC013183208389819A812E
:1015C0002D813E81FC013383228389819A812EE122
:1015D00030E0FC013583248326960FB6F894DEBFF5
:1015E0000FBECDBFDF91CF910895CF93DF93CDB7DD
:1015F000DEB72A970FB6F894DEBF0FBECDBF9E832D
:101600008D834F83588769877A878D819E81FC01FE
:10161000848195819C01990F440B550B8F8198858E
:10162000A985BA85BC01CD010E941620DA01C90145
:1016300089839A83AB83BC8389819A81AB81BC8186
:101640002D813E81AC01BD01C9010E94300B2A965B
:101650000FB6F894DEBF0FBECDBFDF91CF910895D6
:10166000CF93DF93CDB7DEB728970FB6F894DEBFE0
:101670000FBECDBF9C838B834D835E836F83788742
:101680008B819C81DC0116961C928B819C81FC01D4
:1016900017828B819C81DC0118961C928B819C8126
:1016A000FC0111868D819E81AF81B8858B2F992792
:1016B000AA27BB27282F8B819C81DC011A962C93AB
:1016C0008D819E81AF81B885CD01BB2797FDB095F7
:1016D000AB2F282F8B819C81FC0123878D819E81DC
:1016E000AF81B885892F9A2FAB2FBB27A7FDBA955D
:1016F000282F8B819C81DC011C962C932D818B8162
:101700009C81FC0125878B819C81DC0112962D91A7
:101710003C918B819C81FC0180819181A901BC015C
:101720008DED91E00E9422118091DD019091DE010A
:101730000296DC012D913C918B819C81069648E0BC
:1017400050E0BC018DED91E0F90109958DED91E03E
:101750000E94B1119C018B819C81DC011F963C93FE
:101760002E931E978B819C81FC01868597854396DD
:10177000DC018C91882F90E09C012F7033278B81A6
:101780009C81FC01318B208B8B819C81DC015296EA
:101790001D921D921D921C9255971A821982898161
:1017A0009A8104970CF043C08B819C81FC01828953
:1017B0009389A489B589BA2FA92F982F88272B81BF
:1017C0003C81F901828B938BA48BB58B8B819C819F
:1017D000DC0152962D913D914D915C9155978B81F5
:1017E0009C81FC01868597856B817C81DB0150960D
:1017F000ED91FC9169817A816E0F7F1F860F971F93
:10180000FC018081882F90E0A0E0B0E0822B932B38
:10181000A42BB52B2B813C81F901828B938BA48B5C
:10182000B58B89819A8101969A838983B8CF8B8100
:101830009C81FC0182899389A489B589BF772B811A
:101840003C81F901828B938BA48BB58B8B819C811E
:10185000FC0182899389A489B58920E432E44FE0B0
:1018600050E0BC01CD010E941620DC01CB012B8190
:101870003C81F901828B938BA48BB58B8B819C81EE
:10188000FC0182899389A489B5892B813C812A5ED8
:101890003F4F4B2F4F934A2F4F93492F4F938F9387
:1018A00084E991E0892F8F9384E991E08F93832FCE
:1018B0008F93822F8F930E9487208DB79EB70896B3
:1018C0000FB6F894DEBF0FBECDBF8B819C814696CC
:1018D00028960FB6F894DEBF0FBECDBFDF91CF9133
:1018E0000895CF93DF9300D0CDB7DEB79A83898375
:1018F0002EE731E089819A81FC013183208389813F
:101900009A81FC01138212820F900F90DF91CF9188
:101910000895CF93DF9300D0CDB7DEB79A83898344
:1019200080E090E00F900F90DF91CF910895CF93DA
:10193000DF9300D0CDB7DEB79A8389830F900F90E5
:10194000DF91CF910895CF93DF9300D0CDB7DEB76D
:101950009A83898389819A818B5B9F4F24E1E0E39D
:10196000F1E0DC0101900D922A95E1F789819A81DD
:10197000875A9F4FFC011082118212821382898143
:101980009A818C5B9F4FFC0110820F900F90DF912A
:10199000CF910895CF93DF9300D000D000D01F9255
:1019A000CDB7DEB79A8389834B835C836D837E8357
:1019B0002F838F81682F70E08B819C81AD81BE81E8
:1019C0009C01AD01062E04C0220F331F441F551F7A
:1019D0000A94D2F77195619571096F71772704C0E8
:1019E000B695A795979587956A95D2F7822B932BF5
:1019F000A42BB52BBC01CD0127960FB6F894DEBF02
:101A00000FBECDBFDF91CF910895EF92FF920F935C
:101A10001F93CF93DF93CDB7DEB76B970FB6F894D4
:101A2000DEBF0FBECDBF9B8F8A8F8A8D9B8D8B5B58
:101A30009F4FFC0180819181A281B3818A839B8326
:101A4000AC83BD838A8D9B8D875B9F4FFC0180811A
:101A50009181A281B3818E839F83A887B9878A8D64
:101A60009B8D835B9F4FFC0180819181A281B3811B
:101A70008A879B87AC87BD878A8D9B8D8F5A9F4FA6
:101A8000FC0180819181A281B3818E879F87A88B81
:101A9000B98B8A8D9B8D8B5A9F4FFC0180819181E0
:101AA000A281B3818A8B9B8BAC8BBD8B1982898180
:101AB000803508F08AC18981803108F483C089812A
:101AC000882F90E00D968F7099272A8D3B8D019677
:101AD000880F991F880F991F820F931FFC01208187
:101AE0003181428153818981882F90E008968F70DF
:101AF00099276A8D7B8D0196880F991F880F991FF2
:101B0000860F971FFC0180819181A281B3812827D4
:101B100039274A275B278981882F90E002968F70AA
:101B200099276A8D7B8D0196880F991F880F991FC1
:101B3000860F971FFC0180819181A281B3812827A4
:101B400039274A275B278981882F90E08F70992752
:101B50006A8D7B8D0196880F991F880F991F860FBC
:101B6000971FFC0180819181A281B38182279327F5
:101B7000A427B5278E8B9F8BA88FB98F8981882F3B
:101B800090E08C010F7011278E899F89A88DB98DE7
:101B9000EA8DFB8D21E0AC01BD01CF010E94CA0C92
:101BA000DC01CB014A8D5B8D98012F5F3F4F220FE7
:101BB000331F220F331F240F351FF90180839183B8
:101BC000A283B3838981843128F52A853B854C859E
:101BD0005D858E859F85A889B989282739274A2759
:101BE0005B278E819F81A885B985282339234A23C5
:101BF0005B238E859F85A889B98982279327A4278F
:101C0000B52787569648AD47B54A8E8B9F8BA88FD0
:101C1000B98F6CC089818832E8F42E813F81488574
:101C200059858A859B85AC85BD85282739274A2714
:101C30005B278E859F85A889B98982279327A4274A
:101C4000B5278F559441A642B1498E8B9F8BA88FA3
:101C5000B98F4CC089818C3368F52E813F814885CE
:101C600059858A859B85AC85BD85282339234A23E0
:101C70005B23EE80FF80088519858A859B85AC856E
:101C8000BD85E82AF92A0A2B1B2B8E859F85A889FA
:101C9000B9898E219F21A023B123822B932BA42BC2
:101CA000B52B84529344A44EB0478E8B9F8BA88F44
:101CB000B98F1CC02E813F81488559858A859B85B7
:101CC000AC85BD85282739274A275B278E859F85C8
:101CD000A889B98982279327A427B5278A529E43CA
:101CE000AD49B5438E8B9F8BA88FB98F8A819B811D
:101CF000AC81BD81EA8DFB8D25E0AC01BD01CF013A
:101D00000E94CA0C9B01AC018A899B89AC89BD8960
:101D1000280F391F4A1F5B1F8981882F90E08F7021
:101D200099276A8D7B8D0196880F991F880F991FBF
:101D3000860F971FFC0180819181A281B381820F60
:101D4000931FA41FB51F2E893F89488D598D820F7F
:101D5000931FA41FB51F8E8B9F8BA88FB98F8E8565
:101D60009F85A889B9898A8B9B8BAC8BBD8B8A8513
:101D70009B85AC85BD858E879F87A88BB98B8E810F
:101D80009F81A885B985EA8DFB8D2EE1AC01BD014F
:101D9000CF010E94CA0CDC01CB018A879B87AC87EC
:101DA000BD878A819B81AC81BD818E839F83A887FB
:101DB000B9878E899F89A88DB98D8A839B83AC83CF
:101DC000BD8389818F5F898372CE8A8D9B8D8B5B6A
:101DD0009F4FFC0120813181428153818A819B8107
:101DE000AC81BD81820F931FA41FB51F2A8D3B8D2F
:101DF0002B5B3F4FF90180839183A283B3838A8D4C
:101E00009B8D875B9F4FFC012081318142815381F3
:101E10008E819F81A885B985820F931FA41FB51F4E
:101E20002A8D3B8D275B3F4FF90180839183A283ED
:101E3000B3838A8D9B8D835B9F4FFC012081318111
:101E4000428153818A859B85AC85BD85820F931F16
:101E5000A41FB51F2A8D3B8D235B3F4FF901808363
:101E60009183A283B3838A8D9B8D8F5A9F4FFC01F0
:101E700020813181428153818E859F85A889B989CE
:101E8000820F931FA41FB51F2A8D3B8D2F5A3F4FE2
:101E9000F90180839183A283B3838A8D9B8D8B5AB2
:101EA0009F4FFC0120813181428153818A899B8926
:101EB000AC89BD89820F931FA41FB51F2A8D3B8D4E
:101EC0002B5A3F4FF90180839183A283B3836B9692
:101ED0000FB6F894DEBF0FBECDBFDF91CF911F913B
:101EE0000F91FF90EF900895CF93DF9300D01F9252
:101EF000CDB7DEB79A8389836B8389819A818C5BA6
:101F00009F4FFC01908183E08927882F90E02981F1
:101F10003A81820F931F04962B81FC0120838981D3
:101F20009A818C5B9F4FFC01808121E0280F898181
:101F30009A818C5B9F4FFC01208389819A818C5B05
:101F40009F4FFC018081803451F489819A810E94E5
:101F5000050D89819A818C5B9F4FFC0110820F9047
:101F60000F900F90DF91CF910895CF93DF9300D022
:101F70001F92CDB7DEB79A8389836B8389819A815B
:101F8000875A9F4FFC0180819181A281B381019684
:101F9000A11DB11D29813A81275A3F4FF901808344
:101FA0009183A283B38389819A816B810E94740F8C
:101FB00081E090E00F900F900F90DF91CF91089506
:101FC000CF93DF9300D0CDB7DEB79A838983898121
:101FD0009A8160E80E94740F89819A818C5B9F4F7F
:101FE000FC018081883331F089819A8160E00E9410
:101FF000740FF2CF89819A8160E00E94740F898109
:102000009A8160E00E94740F89819A8160E00E9449
:10201000740F89819A81875A9F4FFC018081918139
:10202000A281B381072E7DE1B695A79597958795F7
:102030007A95D1F7702D282F89819A81622F0E947D
:10204000740F89819A81875A9F4FFC018081918109
:10205000A281B381072E75E1B695A79597958795CF
:102060007A95D1F7702D282F89819A81622F0E944D
:10207000740F89819A81875A9F4FFC0180819181D9
:10208000A281B381072E7DE0B695A7959795879598
:102090007A95D1F7702D282F89819A81622F0E941D
:1020A000740F89819A81875A9F4FFC0180819181A9
:1020B000A281B381689414F8B695A79597958795F2
:1020C0001694D1F7282F89819A81622F0E94740F6C
:1020D00089819A81875A9F4FFC0180819181A281D9
:1020E000B381282F220F220F220F89819A81622F1C
:1020F0000E94740F0F900F90DF91CF910895CF93AE
:10210000DF93CDB7DEB72C970FB6F894DEBF0FBEC6
:10211000CDBF9C878B878B859C850E94E00F1A82A0
:10212000198289819A8105970CF07FC02B853C85A7
:1021300089819A81880F991F880F991F820F931F99
:102140008B5B9F4FFC0180819181A281B3818B8346
:102150009C83AD83BE838B819C81AD81BE81B82F72
:10216000AA27992788278F839887A987BA878B8181
:102170009C81AD81BE81BA2FA92F982F88278827EF
:102180009927BB272F81388549855A85822B932B28
:10219000A42BB52B8F839887A987BA878B819C81C5
:1021A000AD81BE81892F9A2FAB2FBB278827AA2705
:1021B000BB272F81388549855A85822B932BA42BE9
:1021C000B52B8F839887A987BA878B819C81AD8136
:1021D000BE818B2F9927AA27BB272F813885498558
:1021E0005A85822B932BA42BB52B8F839887A98795
:1021F000BA872B853C8589819A81880F991F880F22
:10220000991F820F931F9C012B5B3F4F8F819885F5
:10221000A985BA85F90180839183A283B3838981DB
:102220009A8101969A8389837CCF8B859C858B5B71
:102230009F4F2C960FB6F894DEBF0FBECDBFDF9137
:10224000CF910895CF93DF9300D000D000D01F929C
:10225000CDB7DEB79B838A837D836C835F834E8398
:102260008A819B81835A9F4F40E450E060E070E098
:102270000E9477208E819F8181349105BCF18A81F3
:102280009B810E94A30C8E819F819C01215031096A
:102290003F832E8321E0892B09F420E02223B9F02B
:1022A0008A819B81FC0180819181FC0120813181A7
:1022B0008C819D81AC014F5F5F4F5D834C83FC013E
:1022C00040818A819B81642FF9010995DCCF8A8145
:1022D0009B810E947F109C018A819B81835A9F4F22
:1022E00044E150E0B9010E946E200BC04E815F8135
:1022F0008A819B81835A9F4F2C813D81B9010E9425
:102300006E208A819B810E94A30C1982898180346E
:10231000F8F48A819B81FC0180819181FC012081FC
:1023200031818981882F90E04A815B81840F951FDC
:10233000835A9F4FFC01908186E3492F48278A8169
:102340009B81642FF901099589818F5F8983DECF95
:1023500027960FB6F894DEBF0FBECDBFDF91CF91A9
:102360000895CF93DF9300D01F92CDB7DEB79B8344
:102370008A838A819B810E947F109C018A819B8134
:1023800083569F4F44E150E0B9010E946E208A813C
:102390009B810E94A30C198289818034F8F48A8180
:1023A0009B81FC0180819181FC01208131818981A7
:1023B000882F90E04A815B81840F951F835A9F4F3D
:1023C000FC0190818CE5492F48278A819B81642FED
:1023D000F901099589818F5F8983DECF198289810F
:1023E0008431E0F48A819B81FC0180819181FC0130
:1023F000208131818981882F90E04A815B81840F1F
:10240000951F83569F4FFC0140818A819B81642FD9
:10241000F901099589818F5F8983E1CF8A819B8149
:102420000E947F100F900F900F90DF91CF91089531
:10243000CF93DF9300D0CDB7DEB79A8389838981AC
:102440009A810E94710C28E431E089819A81FC0113
:10245000318320830F900F90DF91CF910895CF9318
:10246000DF9300D000D0CDB7DEB79A8389837C8319
:102470006B8389819A81019741F48B819C810196BC
:1024800021F48DED91E00E9418120F900F900F90A3
:102490000F90DF91CF910895CF93DF93CDB7DEB743
:1024A0006FEF7FEF81E090E00E942F12DF91CF91DC
:1024B00008951F920F920FB60F9211248F939F933E
:1024C000AF93BF93CF93DF93CDB7DEB72597DEBF32
:1024D000CDBF8091920290919302A0919402B0910D
:1024E000950289839A83AB83BC83809196028D8306
:1024F00089819A81AB81BC810196A11DB11D89831F
:102500009A83AB83BC838D818D5F8D838D818D3765
:1025100070F08D818D578D8389819A81AB81BC81CB
:102520000196A11DB11D89839A83AB83BC838D81E4
:102530008093960289819A81AB81BC8180939202BB
:1025400090939302A0939402B093950280918E028F
:1025500090918F02A0919002B09191020196A11DDD
:10256000B11D80938E0290938F02A0939002B0933E
:1025700091020F900F900F900F900F90DF91CF91DD
:10258000BF91AF919F918F910F900FBE0F901F90B1
:102590001895CF93DF9300D000D01F92CDB7DEB750
:1025A0008FE590E0FC0180818983F894809192020C
:1025B00090919302A0919402B09195028A839B839B
:1025C000AC83BD838FE590E02981FC0120838A8163
:1025D0009B81AC81BD81BC01CD010F900F900F900C
:1025E0000F900F90DF91CF910895CF93DF9300D09C
:1025F00000D000D0CDB7DEB78FE590E0FC01808140
:102600008D83F89480918E0290918F02A091900218
:10261000B091910289839A83AB83BC8386E490E076
:10262000FC0180818E8385E390E0FC018081882F0E
:1026300090E081709927892B71F08E818F3F59F03E
:1026400089819A81AB81BC810196A11DB11D8983CD
:102650009A83AB83BC838FE590E02D81FC012083BE
:1026600089819A81AB81BC812227382F492F5A2F2B
:102670008E81882F90E0A0E0B0E0820F931FA41F0E
:10268000B51F880F991FAA1FBB1F880F991FAA1F6C
:10269000BB1FBC01CD0126960FB6F894DEBF0FBE5E
:1026A000CDBFDF91CF910895EF92FF920F931F93CB
:1026B000CF93DF93CDB7DEB728970FB6F894DEBF80
:1026C0000FBECDBF6D837E838F8398870E94F512E6
:1026D000DC01CB0189839A83AB83BC8337C00E9422
:1026E000861D17C08D819E81AF81B8850197A10994
:1026F000B1098D839E83AF83B88789819A81AB812D
:10270000BC8188519C4FAF4FBF4F89839A83AB8365
:10271000BC838D819E81AF81B885892B8A2B8B2BC1
:10272000A9F00E94F5129B01AC0189819A81AB81CD
:10273000BC8179018A01E81AF90A0A0B1B0BD8013E
:10274000C701883E9340A105B10560F68D819E8149
:10275000AF81B885892B8A2B8B2B09F628960FB66B
:10276000F894DEBF0FBECDBFDF91CF911F910F91C7
:10277000FF90EF900895CF93DF9300D0CDB7DEB7F1
:102780009A83898389819A81029798F089819A81B5
:10279000880F991F880F991F9A83898389819A814D
:1027A00005979A83898389819A810197F1F79A83A2
:1027B00089830F900F90DF91CF910895CF93DF938E
:1027C000CDB7DEB7789484E490E0FC01208184E406
:1027D00090E02260FC01208384E490E0FC012081F1
:1027E00084E490E02160FC01208385E490E0FC011A
:1027F000208185E490E02260FC01208385E490E064
:10280000FC01208185E490E02160FC0120838EE6BC
:1028100090E0FC0120818EE690E02160FC012083A5
:1028200081E890E0FC01108281E890E0FC012081C9
:1028300081E890E02260FC01208381E890E0FC01C7
:10284000208181E890E02160FC01208380E890E015
:10285000FC01208180E890E02160FC01208381EB75
:1028600090E0FC01208181EB90E02460FC0120835A
:1028700080EB90E0FC01208180EB90E02160FC0186
:1028800020838AE790E0FC0120818AE790E02460C1
:10289000FC0120838AE790E0FC0120818AE790E038
:1028A0002260FC0120838AE790E0FC0120818AE716
:1028B00090E02160FC0120838AE790E0FC01208108
:1028C0008AE790E02068FC01208381EC90E0FC0125
:1028D0001082DF91CF910895CF93DF93CDB7DEB70C
:1028E00069970FB6F894DEBF0FBECDBF888F698F92
:1028F000888D882F90E086569F4F9A83898389819F
:102900009A81FC0184918B838B818C83888D882FA5
:1029100090E08A579F4F9E838D838D819E81FC011D
:1029200084918F838F8188878885882309F494C058
:102930008885882F90E0880F991F88599F4F9A8724
:10294000898789859A85FC0125913491CF013C873F
:102950002B879A8789878B859C859E878D8788851D
:10296000882F90E0880F991F8E589F4F988B8F87E4
:102970008F859889FC0125913491CF013A8B298B61
:10298000988B8F8789899A899C8B8B8B898D8823DB
:1029900031F58FE590E0FC0180818F8BF8948D8577
:1029A0009E85FC018081982F8C8180958923282F1A
:1029B0008D859E85FC0120838B899C89FC0180810B
:1029C000982F8C8180958923282F8B899C89FC01E5
:1029D00020838FE590E02F89FC0120833DC0898D05
:1029E000823021F58FE590E0FC0180818E8BF89498
:1029F0008D859E85FC018081982F8C81809589230F
:102A0000282F8D859E85FC0120838B899C89FC0164
:102A100090818C81292F282B8B899C89FC01208314
:102A20008FE590E02E89FC01208316C08FE590E0B1
:102A3000FC0180818D8BF8948D859E85FC019081B1
:102A40008C81292F282B8D859E85FC0120838FE585
:102A500090E02D89FC01208369960FB6F894DEBFC3
:102A60000FBECDBFDF91CF910895CF93DF931F921B
:102A7000CDB7DEB789838981882F90E083309105B7
:102A800091F08430910534F48130910501F1029781
:102A900041F144C08730910571F188309105A9F169
:102AA000049759F03BC080E890E0FC01208180E869
:102AB00090E02F77FC01208331C080E890E0FC019A
:102AC000208180E890E02F7DFC01208327C084E4F2
:102AD00090E0FC01208184E490E02F77FC012083CA
:102AE0001DC084E490E0FC01208184E490E02F7D0F
:102AF000FC01208313C080EB90E0FC01208180EB7F
:102B000090E02F77FC01208309C080EB90E0FC016E
:102B1000208180EB90E02F7DFC0120830F90DF91DE
:102B2000CF910895CF93DF93CDB7DEB765970FB6FA
:102B3000F894DEBF0FBECDBF8C8B6D8B8C89882F38
:102B400090E082559F4F9A83898389819A81FC0105
:102B500084918B838B818C838C89882F90E086561F
:102B60009F4F9E838D838D819E81FC0184918F83F5
:102B70008F8188878C89882F90E08A579F4F9A870A
:102B8000898789859A85FC0184918B878B858C87C1
:102B90008C85882309F444C08C81882319F08C81AA
:102BA0000E9435158C85882F90E0880F991F8E58CC
:102BB0009F4F9E878D878D859E85FC012591349141
:102BC000CF01388B2F879E878D878F8598899A8B29
:102BD000898B8FE590E0FC0180818B8BF8948D8947
:102BE000882371F489899A89FC018081982F8885CE
:102BF00080958923282F89899A89FC0120830BC01D
:102C000089899A89FC0190818885292F282B8989B7
:102C10009A89FC0120838FE590E02B89FC012083B9
:102C200065960FB6F894DEBF0FBECDBFDF91CF9192
:102C30000895CF93DF93CDB7DEB761970FB6F894C1
:102C4000DEBF0FBECDBF898B8989882F90E082556A
:102C50009F4F9A83898389819A81FC0184918B8318
:102C60008B818C838989882F90E086569F4F9E8325
:102C70008D838D819E81FC0184918F838F818887D4
:102C80008989882F90E08A579F4F9A8789878985FD
:102C90009A85FC0184918B878B858C878C85882312
:102CA00019F480E090E026C08C81882319F08C8193
:102CB0000E9435158C85882F90E0880F991F8458C5
:102CC0009F4F9E878D878D859E85FC012591349130
:102CD000CF01388B2F879E878D878F859889FC0140
:102CE000908188858923882319F081E090E002C0D3
:102CF00080E090E061960FB6F894DEBF0FBECDBFC6
:102D0000DF91CF910895CF93DF9300D0CDB7DEB799
:102D10009A83898389819A81FC01848195810F90AE
:102D20000F90DF91CF910895CF93DF9300D0CDB76F
:102D3000DEB79A83898389819A81FC0180819181A0
:102D40000F900F90DF91CF9108950F931F93CF9322
:102D5000DF9300D000D0CDB7DEB79A8389837C8320
:102D60006B838B819C81892B19F480E090E015C0E6
:102D700089819A81FC01808191810296FC01008108
:102D800011818B819C810E947E20AC012B813C8132
:102D900089819A81B901F80109950F900F900F90E0
:102DA0000F90DF91CF911F910F910895CF93DF93F3
:102DB00000D000D000D0CDB7DEB79A8389837C8362
:102DC0006B835E834D8389819A81FC01808191812F
:102DD0000296FC01208131814D815E816B817C8175
:102DE00089819A81F901099526960FB6F894DEBF7C
:102DF0000FBECDBFDF91CF910895CF93DF93CDB7B5
:102E0000DEB728970FB6F894DEBF0FBECDBF9C8308
:102E10008B837E836D8358874F831A8219828F81BB
:102E200098859C012150310938872F8321E0892B17
:102E300009F420E0222311F18B819C81FC01808127
:102E40009181FC01208131818D819E81AC014F5F98
:102E50005F4F5E834D83FC0140818B819C81642F99
:102E6000F901099521E0892B09F420E0222331F0B2
:102E700089819A8101969A838983D1CF89819A81A8
:102E800028960FB6F894DEBF0FBECDBFDF91CF916D
:102E90000895CF93DF93CDB7DEB72C970FB6F89494
:102EA000DEBF0FBECDBF9A8789877C876B878B85F6
:102EB0009C859A8389831C821B8289819A819C01CB
:102EC0002F5F3F4F3A8329839E838D838D819E811F
:102ED000FC0184918F838F81888788858823C9F03E
:102EE00089859A85FC0180819181FC012081318155
:102EF00089859A856885F901099521E0892B09F46E
:102F000020E0222331F08B819C8101969C838B836E
:102F1000D4CF8B819C812C960FB6F894DEBF0FBE68
:102F2000CDBFDF91CF9108950F931F93CF93DF9380
:102F300000D000D0CDB7DEB79A8389837C836B83C2
:102F40008B819C810E9483168C018B819C810E94C5
:102F500094169C0189819A81A801B9010E94D61614
:102F60000F900F900F900F90DF91CF911F910F91C5
:102F70000895CF93DF9300D000D0CDB7DEB79A830A
:102F800089837C836B832B813C8189819A81B90100
:102F90000E94A5160F900F900F900F90DF91CF9188
:102FA0000895CF93DF9300D01F92CDB7DEB79A83F9
:102FB00089836B8389819A81FC0180819181FC01E5
:102FC000208131814B8189819A81642FF901099592
:102FD0000F900F900F90DF91CF910895CF93DF93D3
:102FE00000D000D01F92CDB7DEB79A8389836B8360
:102FF0005D834C838B81882F90E0A0E0B0E02C8132
:103000003D81E981FA81AC01BD01CF010E94D21856
:103010000F900F900F900F900F90DF91CF91089528
:10302000CF93DF9300D000D000D0CDB7DEB79A8326
:1030300089837C836B835E834D838B819C81092E86
:10304000000CAA0BBB0B2D813E81E981FA81AC01FA
:10305000BD01CF010E94591826960FB6F894DEBF25
:103060000FBECDBFDF91CF910895CF93DF9300D0F6
:1030700000D000D0CDB7DEB79A8389837C836B8381
:103080005E834D838B819C81CC01A0E0B0E02D81DB
:103090003E81E981FA81AC01BD01CF010E94D218C5
:1030A00026960FB6F894DEBF0FBECDBFDF91CF914D
:1030B0000895CF93DF93CDB7DEB72A970FB6F89474
:1030C000DEBF0FBECDBF9C838B834D835E836F833A
:1030D00078873A87298789859A85892B79F48B8126
:1030E0009C81FC0180819181FC01208131814D8195
:1030F0008B819C81642FF90109954BC089859A8544
:103100000A97D9F58D819E81AF81B885BB2344F59F
:103110008B819C816DE20E94D1179A8389838D8176
:103120009E81AF81B885B095A095909581959F4F70
:10313000AF4FBF4F8D839E83AF83B8878D819E81B4
:10314000AF81B885EB81FC812AE0AC01BD01CF01E4
:103150000E94671B9C0189819A81820F931F19C06D
:103160008D819E81AF81B885EB81FC812AE0AC0125
:10317000BD01CF010E94671B0CC029858D819E81F6
:10318000AF81B885EB81FC81AC01BD01CF010E940C
:10319000671B2A960FB6F894DEBF0FBECDBFDF9136
:1031A000CF910895CF93DF93CDB7DEB728970FB6B1
:1031B000F894DEBF0FBECDBF9A8389834B835C83B7
:1031C0006D837E8338872F838F819885892B79F44F
:1031D00089819A81FC0180819181FC01208131816A
:1031E0004B8189819A81642FF90109950CC02F8147
:1031F0008B819C81AD81BE81E981FA81AC01BD01E9
:10320000CF010E94671B28960FB6F894DEBF0FBE51
:10321000CDBFDF91CF910895CF93DF93CDB7DEB7C8
:1032200028970FB6F894DEBF0FBECDBF9A8389836F
:103230004B835C836D837E8338872F832F818B81C3
:103240009C81AD81BE81E981FA81AC01BD01CF01D4
:103250000E94D41B28960FB6F894DEBF0FBECDBFD8
:10326000DF91CF910895CF93DF9300D000D000D0AD
:10327000CDB7DEB79C838B837E836D832D813E81AA
:103280008B819C81B9010E9449179A8389838B8124
:103290009C810E947D199C0189819A81820F931FD4
:1032A0009A83898389819A8126960FB6F894DEBF26
:1032B0000FBECDBFDF91CF910895CF93DF9300D0A4
:1032C00000D0CDB7DEB79A8389837C836B838B81F3
:1032D0009C81FC0180819181FC01208131814981A7
:1032E0005A818B819C81BA01F90109950F900F9049
:1032F0000F900F90DF91CF910895CF93DF9300D07F
:10330000CDB7DEB79A83898389819A816AE971E0B2
:103310000E94A5160F900F90DF91CF910895CF9343
:10332000DF9300D000D000D0CDB7DEB79C838B8375
:103330007E836D832D813E818B819C81B9010E94AA
:1033400094179A8389838B819C810E947D199C01AB
:1033500089819A81820F931F9A83898389819A81B7
:1033600026960FB6F894DEBF0FBECDBFDF91CF918A
:103370000895CF93DF9300D000D000D0CDB7DEB753
:103380009C838B837E836D832D813E818B819C8189
:10339000B9010E94B9179A8389838B819C810E940D
:1033A0007D199C0189819A81820F931F9A83898359
:1033B00089819A8126960FB6F894DEBF0FBECDBFE5
:1033C000DF91CF910895CF93DF9300D000D01F926B
:1033D000CDB7DEB79C838B836D838B819C816D81A0
:1033E0000E94D1179A8389838B819C810E947D19C9
:1033F0009C0189819A81820F931F9A838983898195
:103400009A810F900F900F900F900F90DF91CF91B6
:103410000895CF93DF9300D000D000D01F92CDB796
:10342000DEB79C838B836D835F834E832E813F81C8
:103430008B819C81A9016D810E94EE179A838983FB
:103440008B819C810E947D199C0189819A81820FC8
:10345000931F9A83898389819A8127960FB6F8945E
:10346000DEBF0FBECDBFDF91CF910895CF93DF9325
:10347000CDB7DEB728970FB6F894DEBF0FBECDBF2D
:103480009C838B837E836D8358874F834F815885C0
:103490002D813E818B819C81B9010E9410189A83F5
:1034A00089838B819C810E947D199C0189819A81ED
:1034B000820F931F9A83898389819A8128960FB6F8
:1034C000F894DEBF0FBECDBFDF91CF910895CF93AB
:1034D000DF93CDB7DEB728970FB6F894DEBF0FBEE7
:1034E000CDBF9C838B837E836D8358874F834F81B1
:1034F00058852D813E818B819C81B9010E943518B0
:103500009A8389838B819C810E947D199C0189818A
:103510009A81820F931F9A83898389819A81289641
:103520000FB6F894DEBF0FBECDBFDF91CF910895E7
:10353000CF93DF93CDB7DEB72A970FB6F894DEBFEF
:103540000FBECDBF9C838B834D835E836F83788753
:103550003A87298729853A858D819E81AF81B885F3
:10356000EB81FC81AC01BD01CF010E9459189A8307
:1035700089838B819C810E947D199C0189819A811C
:10358000820F931F9A83898389819A812A960FB625
:10359000F894DEBF0FBECDBFDF91CF910895CF93DA
:1035A000DF93CDB7DEB72A970FB6F894DEBF0FBE14
:1035B000CDBF9C838B834D835E836F8378873A87EF
:1035C000298729853A858D819E81AF81B885EB81D8
:1035D000FC81AC01BD01CF010E94D2189A8389837E
:1035E0008B819C810E947D199C0189819A81820F27
:1035F000931F9A83898389819A812A960FB6F894BA
:10360000DEBF0FBECDBFDF91CF910895CF93DF9383
:10361000CDB7DEB72A970FB6F894DEBF0FBECDBF89
:103620009C838B834D835E836F8378873A8729875A
:1036300029853A858D819E81AF81B885EB81FC819A
:10364000AC01BD01CF010E940C199A8389838B8143
:103650009C810E947D199C0189819A81820F931F10
:103660009A83898389819A812A960FB6F894DEBF5E
:103670000FBECDBFDF91CF910895CF93DF9300D0E0
:1036800000D000D0CDB7DEB79C838B837E836D8363
:103690002D813E818B819C81B9010E945D199A83A5
:1036A00089838B819C810E947D199C0189819A81EB
:1036B000820F931F9A83898389819A8126960FB6F8
:1036C000F894DEBF0FBECDBFDF91CF910895CF93A9
:1036D000DF93CDB7DEB7AB970FB6F894DEBF0FBE62
:1036E000CDBF9EA38DA34FA358A769A77AA72BA7E9
:1036F000CE01049680969A83898389819A81FC0100
:1037000010828BA5823010F48AE08BA78BA5282F1E
:1037100030E040E050E08FA198A5A9A5BAA5BC0172
:10372000CD010E94F41FDC01CB018B838BA5282FD8
:1037300030E040E050E08FA198A5A9A5BAA5BC0152
:10374000CD010E94F41FDA01C9018FA398A7A9A790
:10375000BAA78B818A3024F48B81805D282F03C027
:103760008B81895C282F89819A8101979A8389832B
:1037700089819A81FC0120838FA198A5A9A5BAA56A
:10378000892B8A2B8B2B11F629813A818DA19EA141
:10379000B9010E94A516AB960FB6F894DEBF0FBE16
:1037A000CDBFDF91CF910895CF92DF92EF92FF923C
:1037B0001F93CF93DF93CDB7DEB768970FB6F8941A
:1037C000DEBF0FBECDBF9B8B8A8B4C8B5D8B6E8B10
:1037D0007F8B288F1A8219822C893D894E895F89B7
:1037E0006C897D898E899F890E94CB1F882311F067
:1037F00081E001C080E0882339F08A899B896DE9E6
:1038000071E00E94B91739C18C899D89AE89BF8941
:103810006C017D01E894F7F811E02FEF3FEF4FE7DF
:103820005FE7C701B6010E94CB1F882359F42FEF31
:103830003FEF4FE75FE7C701B6010E94FA1D181678
:103840000CF410E081E08127882F90E081708823BC
:1038500039F08A899B8961EA71E00E94B9170DC12C
:103860002FEF3FEF4FE75FE46C897D898E899F8959
:103870000E94591F18163CF48A899B8965EA71E0F9
:103880000E94B917FAC02FEF3FEF4FE75FEC6C894A
:103890007D898E899F890E94FA1D88233CF48A893C
:1038A0009B8965EA71E00E94B917E7C020E030E02B
:1038B000A9016C897D898E899F890E94FA1D8823C0
:1038C000ACF48A899B896DE20E94D1179C018981A1
:1038D0009A81820F931F9A8389838C899D89AE89EF
:1038E000BF89B0588C8B9D8BAE8BBF8B80E090E0F6
:1038F000A0E0BFE38B839C83AD83BE831F829F8147
:10390000888D9817A0F420E030E040E251E46B810C
:103910007C818D819E810E94FF1DDC01CB018B8308
:103920009C83AD83BE838F818F5F8F83E8CF2B8194
:103930003C814D815E816C897D898E899F890E9441
:103940008E1DDC01CB018C8B9D8BAE8BBF8B6C896C
:103950007D898E899F890E94781EDC01CB018C872E
:103960009D87AE87BF876C857D858E859F850E94EC
:10397000A71EDC01CB019C01AD016C897D898E897C
:103980009F890E948D1DDC01CB0188879987AA87BA
:10399000BB878C859D85AE85BF85EA89FB892AE03A
:1039A00030E0AC01BD01CF010E94D2189C01898199
:1039B0009A81820F931F9A838983888D882361F06F
:1039C0008A899B896EE20E94D1179C0189819A8124
:1039D000820F931F9A838983888D9FEF980F988F0A
:1039E00091E0882309F490E0992309F444C020E091
:1039F00030E040E251E4688579858A859B850E94A4
:103A00005E1FDC01CB0188879987AA87BB87688501
:103A100079858A859B850E94781EDC01CB01998B74
:103A2000888B288939898A899B894AE050E0B901C5
:103A30000E9435189C0189819A81820F931F9A8375
:103A4000898388899989CC01A0E0B0E0BC01CD01CF
:103A50000E94A71EDC01CB019C01AD016885798520
:103A60008A859B850E948D1DDC01CB018887998703
:103A7000AA87BB87B1CF89819A8168960FB6F894DF
:103A8000DEBF0FBECDBFDF91CF911F91FF90EF90B2
:103A9000DF90CF900895CF93DF93CDB7DEB70E942C
:103AA0006920CF93DF93CDB7DEB70E946920CF9313
:103AB000DF9300D0CDB7DEB79A83898380E090E0B2
:103AC0000F900F90DF91CF910895CF93DF93CDB7F3
:103AD000DEB7DF91CF910895CF93DF93CDB7DEB7F7
:103AE000DF91CF910895CF93DF93CDB7DEB70E94DA
:103AF000DE130E94651D0E9443090E942C0A80E08B
:103B000090E0892BD1F30E940000F7CFCF93DF9391
:103B1000CDB7DEB7DF91CF9108955058BB27AA27C4
:103B20000E94A51D0C941F1F0E94111F38F00E94B7
:103B3000181F20F039F49F3F19F426F40C940E1F3F
:103B40000EF4E095E7FB0C94081FE92F0E94301F4C
:103B500058F3BA17620773078407950720F079F4C2
:103B6000A6F50C94521F0EF4E0950B2EBA2FA02D43
:103B70000B01B90190010C01CA01A0011124FF271A
:103B8000591B99F0593F50F4503E68F11A16F04015
:103B9000A22F232F342F4427585FF3CF4695379514
:103BA0002795A795F0405395C9F77EF41F16BA0BD9
:103BB000620B730B840BBAF09150A1F0FF0FBB1F87
:103BC000661F771F881FC2F70EC0BA0F621F731FD0
:103BD000841F48F4879577956795B795F7959E3F2D
:103BE00008F0B0CF9395880F08F09927EE0F9795BE
:103BF000879508950E94E41E08F481E008950E94CC
:103C0000131E0C941F1F0E94181F58F00E94111FB2
:103C100040F029F45F3F29F00C94081F51110C94D7
:103C2000531F0C940E1F0E94301F68F39923B1F3A9
:103C3000552391F3951B550BBB27AA2762177307D2
:103C4000840738F09F5F5F4F220F331F441FAA1F66
:103C5000A9F335D00E2E3AF0E0E832D09150504022
:103C6000E695001CCAF72BD0FE2F29D0660F771FD0
:103C7000881FBB1F261737074807AB07B0E809F0B6
:103C8000BB0B802DBF01FF2793585F4F3AF09E3F3B
:103C9000510578F00C94081F0C94531F5F3FE4F318
:103CA000983ED4F3869577956795B795F7959F5F7E
:103CB000C9F7880F911D9695879597F90895E1E0CA
:103CC000660F771F881FBB1F621773078407BA0729
:103CD00020F0621B730B840BBA0BEE1F88F7E09584
:103CE00008950E94781E6894B1110C94531F089592
:103CF0000E94381F88F09F5798F0B92F9927B75125
:103D0000B0F0E1F0660F771F881F991F1AF0BA957F
:103D1000C9F714C0B13091F00E94521FB1E008956C
:103D20000C94521F672F782F8827B85F39F0B93F5E
:103D3000CCF3869577956795B395D9F73EF4909532
:103D40008095709561957F4F8F4F9F4F0895E894B0
:103D500009C097FB3EF490958095709561957F4FD3
:103D60008F4F9F4F9923A9F0F92F96E9BB27939581
:103D7000F695879577956795B795F111F8CFFAF491
:103D8000BB0F11F460FF1BC06F5F7F4F8F4F9F4FC2
:103D900016C0882311F096E911C0772321F09EE820
:103DA000872F762F05C0662371F096E8862F70E086
:103DB00060E02AF09A95660F771F881FDAF7880F60
:103DC0009695879597F90895990F0008550FAA0BB6
:103DD000E0E8FEEF16161706E807F907C0F012161E
:103DE0001306E407F50798F0621B730B840B950B21
:103DF00039F40A2661F0232B242B252B21F4089576
:103E00000A2609F4A140A6958FEF811D811D089512
:103E100097F99F6780E870E060E008959FEF80EC7D
:103E2000089500240A941616170618060906089520
:103E300000240A9412161306140605060895092E86
:103E40000394000C11F4882352F0BB0F40F4BF2BF5
:103E500011F460FF04C06F5F7F4F8F4F9F4F089535
:103E600057FD9058440F551F59F05F3F71F047952B
:103E7000880F97FB991F61F09F3F79F08795089510
:103E8000121613061406551FF2CF4695F1DF08C02F
:103E9000161617061806991FF1CF8695710561054C
:103EA00008940895E894BB2766277727CB0197F9F4
:103EB00008950E94E41E08F48FEF08950E94711F78
:103EC0000C941F1F0E94111F38F00E94181F20F031
:103ED000952311F00C94081F0C940E1F11240C94C0
:103EE000531F0E94301F70F3959FC1F3950F50E050
:103EF000551F629FF001729FBB27F00DB11D639F9C
:103F0000AA27F00DB11DAA1F649F6627B00DA11D41
:103F1000661F829F2227B00DA11D621F739FB00DE7
:103F2000A11D621F839FA00D611D221F749F332757
:103F3000A00D611D231F849F600D211D822F762FF0
:103F40006A2F11249F5750409AF0F1F088234AF0CD
:103F5000EE0FFF1FBB1F661F771F881F9150504039
:103F6000A9F79E3F510580F00C94081F0C94531F35
:103F70005F3FE4F3983ED4F3869577956795B795C0
:103F8000F795E7959F5FC1F7FE2B880F911D9695DA
:103F9000879597F908950E94E41E880B990B089560
:103FA000DB018F939F930E943520BF91AF91A29F19
:103FB000800D911DA39F900DB29F900D1124089527
:103FC00097FB072E16F4009407D077FD09D00E94C6
:103FD000402007FC05D03EF4909581959F4F0895B1
:103FE000709561957F4F0895A1E21A2EAA1BBB1B05
:103FF000FD010DC0AA1FBB1FEE1FFF1FA217B307B5
:10400000E407F50720F0A21BB30BE40BF50B661FCA
:10401000771F881F991F1A9469F76095709580958E
:1040200090959B01AC01BD01CF010895052E97FB32
:104030001EF400940E942D2057FD07D00E94F41F0B
:1040400007FC03D04EF40C942D20509540953095EC
:1040500021953F4F4F4F5F4F0895909580957095F4
:1040600061957F4F8F4F9F4F08950E945A20A59FC3
:10407000900DB49F900DA49F800D911D1124089563
:10408000AA1BBB1B51E107C0AA1FBB1FA617B7077E
:1040900010F0A61BB70B881F991F5A95A9F780959A
:1040A0009095BC01CD010895EE0FFF1F0590F4918E
:1040B000E02D0994A29FB001B39FC001A39F700D92
:1040C000811D1124911DB29F700D811D1124911D20
:1040D000089581E090E0F8940C945F23FB01DC01EB
:1040E00002C001900D9241505040D8F70895DC0174
:1040F00001C06D9341505040E0F70895FC010190DC
:104100000020E9F7809590958E0F9F1F0895AEE0EF
:10411000B0E0EDE8F0E20C9436230D891E8986E0CC
:104120008C831A8309838FEF9FE79E838D83AE0173
:10413000475E5F4F6F89788DCE0101960E94AA205D
:104140002F813885020F131FF80110822E96E4E0AC
:104150000C945223ABE0B0E0E0EBF0E20C942823A7
:104160007C013B018A01FC0117821682838181FF59
:10417000C8C1CE0101965C01F7019381F30193FD63
:10418000859193FF81913F01882309F453C18532C2
:1041900039F493FD859193FF81913F01853229F494
:1041A000B70190E00E949A22E7CF912C212C312C6C
:1041B000FFE1F31538F08B3211F190F4803209F100
:1041C000833229F137FC3CC020ED280F2A3050F50E
:1041D00036FE20C08AE0989E200D1124922E06C043
:1041E0008D3291F0803371F7689430F8F30193FDCC
:1041F000859193FF81913F018111DACF21C06894AD
:1042000031F8689432F8F2CF689433F8EFCF6894BD
:1042100034F8ECCFEAE02E9E200D1124222E689473
:1042200035F8E4CF8E3229F436FC04C1689436F8B0
:10423000DDCF8C3619F4689437F8D8CF8836B1F2D0
:10424000982F9F7D95549330E0F08336A1F183370A
:10425000C1F1833509F063C02801F2E04F0E511C13
:10426000F801C080D180692D70E036FC02C06FEF8C
:104270007FEFC6010E9484224C01689437F88201C6
:104280000AC00C5F1F4FFFE3F98388248394912CAD
:104290006501E89437F833FE2DC0522C8114910447
:1042A00071F5552009F468CFB70180E290E00E94D3
:1042B0009A225A94F6CFF801808189830E5F1F4FAE
:1042C000E4CF2801F2E04F0E511CF801C080D180EC
:1042D000692D70E036FC02C06FEF7FEFC6010E94CF
:1042E0008F224C018201D5CFB70180E290E00E947D
:1042F0009A222A942814190409F0B0F7CECFF601B7
:1043000037FC859137FE81916F01B70190E00E94E3
:104310009A2251105A94F1E08F1A9108BFCF843637
:1043200019F0893609F077C0F80137FE6BC060815B
:104330007181828193810C5F1F4FF32DFF763F2E99
:1043400097FF09C090958095709561957F4F8F4F2D
:104350009F4F689437F82AE030E0A5010E94CA22F6
:10436000C82ECA188C2C432C36FE0CC0E89440F89A
:10437000C91440F434FE05C032FC03C0F32DFE7EA8
:104380004F2E892C44FE95C0FE01EC0DF11D80815D
:10439000803309F087C0242D297E422E842D887019
:1043A000582E43FC95C040FE8FC09C2C821418F4FC
:1043B0002C0C922C981844FE91C0B70180E390E039
:1043C0000E949A2242FE09C088E790E041FE02C0A6
:1043D00088E590E0B7010E949A22C91408F48AC0C7
:1043E000CA94D12C9FEFC91AD90ACA0CDB1CF6015A
:1043F00082916F01B70190E00E949A22AC14BD0433
:10440000B1F74FCF60817181072E000C880B990B9B
:104410000E5F1F4F92CFD32CE894D4F82AE030E0FF
:10442000853739F1232D297FD22E8F3601F148F4BB
:104430008835A9F0F701868197812B96E2E10C94EB
:104440004423803749F08837A9F7D4FE02C0689426
:10445000D2F820E130E00DC06894D4F8F6CF34FEF5
:1044600003C0822F8660D82E20E132E002C028E00F
:1044700030E0F801D7FE0FC06081718182819381A5
:104480000C5F1F4FA5010E94CA22C82ECA183D2CDE
:10449000E89437F867CF6081718190E080E00E5F2B
:1044A0001F4FF0CF42FC02C0839478CF8394839453
:1044B00075CF842D867809F471CFF6CFB70180E2ED
:1044C00090E00E949A2283948214C0F3512C73CFFF
:1044D000522C5818821408F46ECFF8CF842D8678A9
:1044E00009F47BCF8BE241FE80E247FC8DE2B7010D
:1044F00090E071CFB70180E390E00E949A229A94F5
:104500006CCF8FEF9FEF99CFFC0105906150704009
:104510000110D8F7809590958E0F9F1F0895FC018C
:104520006150704001900110D8F7809590958E0FE2
:104530009F1F08950F931F93CF93DF93182F092F79
:10454000EB018B8181FD09C01FEF0FEF812F902FB1
:10455000DF91CF911F910F91089582FF14C02E819A
:104560003F818C819D81281739073CF4E881F981CE
:10457000CF0101969983888310838E819F81019654
:104580009F838E83E3CFE885F985812F0995892B59
:10459000A1F3DACFFA01AA27283051F1203181F1B5
:1045A000E8946F936E7F6E5F7F4F8F4F9F4FAF4F3B
:1045B000B1E03ED0B4E03CD0670F781F891F9A1F4E
:1045C000A11D680F791F8A1F911DA11D6A0F711D02
:1045D000811D911DA11D20D009F468943F912AE00E
:1045E000269F11243019305D3193DEF6CF010895F6
:1045F000462F4770405D4193B3E00FD0C9F7F6CF27
:10460000462F4F70405D4A3318F0495D31FD4052EE
:10461000419302D0A9F7EACFB4E0A6959795879584
:1046200077956795BA95C9F7009761057105089563
:104630009B01AC010A2E069457954795379527950F
:10464000BA95C9F7620F731F841F951FA01D0895A7
:104650002F923F924F925F926F927F928F929F9292
:10466000AF92BF92CF92DF92EF92FF920F931F9380
:10467000CF93DF93CDB7DEB7CA1BDB0B0FB6F89431
:10468000DEBF0FBECDBF09942A88398848885F8471
:104690006E847D848C849B84AA84B984C884DF80E2
:1046A000EE80FD800C811B81AA81B981CE0FD11DC6
:1046B0000FB6F894DEBF0FBECDBFED010895F8949C
:0246C000FFCF2A
:1046C2001F1C1F1E1F1E1F1F1E1F1E1F6179792008
:1046D2006C6D616F0A0B0C0D12130E0F1011121379
:1046E20014150A0B0C0D12130E0F101112131415C0
:1046F2000123456789ABCDEFFEDCBA9876543210C0
:10470200F0E1D2C300000000B50FFD16890C970C32
:104712000A0B0C0D12130E0F1011121314150A0BA3
:104722000C0D12130E0F1011121314150A0B0C0D8F
:1047320012130E0F101112131415000000004B1D5E
:10474200FD16890C970C0A0B0C0D12130E0F10118B
:10475200121314152530366C64000D0A006E616E5A
:0A47620000696E66006F76660000C5
:00000001FF
